:100000000C9400070C941D070C941D070C941D07FD
:100010000C941D070C941D070C941D070C941D07D0
:100020000C941D070C941D070C941B240C94D723CF
:100030000C9482250C941D070C941D070C941D072D
:100040000C941D070C941D070C941D070C941D07A0
:100050000C941D070C945E250C941D070C941D0731
:100060000C941D070C941D070C941D070C941D0780
:100070000C941D070C941D070C941D070C941D0770
:100080000C941D070C941D070C941D070C941D0760
:100090000C941D070C941D070C941D070C941D0750
:1000A0000C941D070C941D070C941D070631FF09C5
:1000B00074A1010975150026FF00952075088102BD
:1000C000C005010902A10185020901A10005091964
:1000D000012908150025019508750181020501090E
:1000E0003009311581257F9502750881060938157B
:1000F00081257F950175088106050C0A3802158156
:10010000257F950175088106C0C005010980A10100
:10011000850319012AB700150126B700950175104E
:100120008100C0050C0901A101850419012AA00262
:10013000150126A002950175108100C00501090670
:10014000A1018506050719E029E715002501950895
:10015000750181020507190029EF1500250195F0A9
:10016000750181020508190129059505750191029E
:10017000950175039101C00660FF0961A101096243
:10018000150026FF009520750881020963150026D9
:10019000FF00952075089102C005010906A101051F
:1001A0000719E029E71500250195087501810295D9
:1001B00001750881010507190029FF150026FF00B8
:1001C0009506750881000508190129051500250106
:1001D000950575019102950175039101C00000001C
:1001E000000000000000000000000000000000000F
:1001F00000000000000000000000000000000000FF
:10020000007E0F00D4FFFFFFC70000007800000051
:1002100000000000002A2B28000000000000000061
:10022000000000000000000029000000002C1E3427
:1002300020212224342627252E362D3738271E1F2D
:10024000202122232425263333362E37381F040558
:10025000060708090A0B0C0D0E0F101112131415C6
:10026000161718191A1B1C1D2F3130232D350405A4
:10027000060708090A0B0C0D0E0F101112131415A6
:10028000161718191A1B1C1D2F3130354C444542C6
:1002900055473A2064697361626C65642E0A0044B4
:1002A000454255473A20656E61626C65642E0A00CE
:1002B0003F00433E20004F6E6573686F743A2061C3
:1002C00063746976653A2025640A000A0025303295
:1002D0005820006E6B726F5F7265706F72743A2097
:1002E00025303258207C20000A002530325820006A
:1002F0006B6579626F6172645F7265706F72743A78
:100300002025303258207C200073757370656E6430
:10031000696E67206B6579626F6172640D0A000A0D
:10032000002530313662003A200025303258000A6C
:10033000722F632030313233343536373839414209
:10034000434445460A006C65645F7461736B3A20F0
:10035000253032580A006B65796D61705F636F6E8E
:100360006669672E7261773A20253032580A2E73FB
:100370007761705F636F6E74726F6C5F63617073CF
:100380006C6F636B3A2025750A2E636170736C6F16
:10039000636B5F746F5F636F6E74726F6C3A20256E
:1003A000750A2E737761705F6C63746C5F6C677530
:1003B000693A2025750A2E737761705F7263746CD9
:1003C0005F726775693A2025750A2E737761705FD1
:1003D0006C616C745F6C6775693A2025750A2E73C1
:1003E0007761705F72616C745F726775693A20251E
:1003F000750A2E6E6F5F6775693A2025750A2E7330
:100400007761705F67726176655F6573633A202517
:10041000750A2E737761705F6261636B736C6173D1
:10042000685F6261636B73706163653A2025750A6A
:100430002E6E6B726F3A2025750A2E737761705F8E
:100440006573636170655F636170736C6F636B3A52
:100450002025750A0064656275675F636F6E666963
:10046000672E7261773A20253032580A2E656E6108
:10047000626C653A2025750A2E6D61747269783A4E
:100480002025750A2E6B6579626F6172643A2025AA
:10049000750A2E6D6F7573653A2025750A006565BE
:1004A000636F6E6669673A0A64656661756C745F4E
:1004B0006C617965723A2025750A000A092D204D74
:1004C00061676963202D0A443A09446562756720B3
:1004D0004D65737361676520546F67676C650A5873
:1004E0003A094D6174726978204465627567204DE0
:1004F0006F646520546F67676C65202D2053686FAB
:1005000077206B65797072657373657320696E20EF
:100510006D617472697820677269640A4B3A094B9D
:100520006579626F61726420446562756720546FFB
:1005300067676C65202D2053686F77206B65797035
:1005400072657373207265706F72740A4D3A094454
:1005500065627567204D6F75736520546F67676CB2
:10056000650A563A0956657273696F6E0A533A09FD
:100570005374617475730A433A094163746976610F
:10058000746520436F6E736F6C65204D6F64650AF0
:1005900046312D4631303A095377697463682074C7
:1005A0006F204C6179657220302D3920284631301A
:1005B000203D204C30290A302D393A09537769748F
:1005C000636820746F204C6179657220302D390A80
:1005D00047524156453A0953776974636820746FEE
:1005E000204C6179657220302028616C7465726ED0
:1005F000617465290A423A094A756D7020746F204A
:10060000426F6F746C6F616465720A4553433A09B7
:100610004A756D7020746F20426F6F746C6F6164E7
:1006200065722028616C7465726E617465290A4573
:100630003A095072696E7420454550524F4D20530F
:10064000657474696E67730A4241434B535041436A
:10065000453A09436C65617220454550524F4D0A39
:100660004E3A094E4B524F20546F67676C650A0033
:100670000A092D20436F6E736F6C65202D0A455358
:10068000432F713A09717569740A6D3A096D6F7576
:1006900073656B65790A002573000A092D20537470
:1006A00061747573202D0A686F73745F6B6579626E
:1006B0006F6172645F6C65647328293A202530325B
:1006C000580A6B6579626F6172645F70726F746FE4
:1006D000636F6C3A20253032580A6B6579626F611E
:1006E00072645F69646C653A20253032580A6B6524
:1006F000796D61705F636F6E6669672E6E6B726F86
:100700003A20253032580A74696D65725F726561EE
:1007100064333228293A202530386C580A003F00CB
:100720004E4B524F3A206F66660A004E4B524F3A7C
:10073000206F6E0A000A6D6F7573653A206F6666EA
:100740000A000A6D6F7573653A206F6E0A000A6BB6
:100750006579626F6172643A206F66660A000A6B9F
:100760006579626F6172643A206F6E0A000A6D618A
:10077000747269783A206F66660A000A6D61747255
:1007800069783A206F6E0A000A64656275673A20DC
:100790006F66660A000A64656275673A206F6E0AC2
:1007A000000A0A4A756D70696E6720746F20626F67
:1007B0006F746C6F616465722E2E2E2000433E2094
:1007C00000436C656172696E6720454550524F4D1C
:1007D0000A00313A0964656C6179282A31306D73F9
:1007E000293A2025750A323A09696E746572766174
:1007F0006C286D73293A2025750A333A096D6178A2
:100800005F73706565643A2025750A343A09746926
:100810006D655F746F5F6D61783A2025750A353AB2
:1008200009776865656C5F6D61785F737065656495
:100830003A2025750A363A09776865656C5F7469F0
:100840006D655F746F5F6D61783A2025750A007081
:100850003A097072696E742076616C7565730A640A
:100860003A097365742064656661756C74730A7502
:10087000703A092B310A646E3A092D310A6C743AC8
:10088000092B31300A72743A092D31300A4553432D
:100890002F713A09717569740A0A7370656564206D
:1008A0003D2064656C7461202A206D61785F7370EF
:1008B000656564202A2028726570656174202F2088
:1008C00074696D655F746F5F6D6178290A7768651B
:1008D00072652064656C74613A20637572736F721F
:1008E0003D25642C20776865656C3D25640A536559
:1008F0006520687474703A2F2F656E2E77696B6966
:1009000070656469612E6F72672F77696B692F4D0F
:100910006F7573655F6B6579730A004D3E20004DFE
:1009200025753A25733E20003F0A003D2025750AB3
:10093000003F0A0064656661756C74730A00257572
:100940000A003F0A000A092D2056616C7565732064
:100950002D0A00710A000A092D204D6F7573656B11
:100960006579202D0A004C25640A0035001E001F01
:10097000002000210022002300240025002600275B
:10098000002A002B0014001A000800150017001C94
:100990000018000C00120013004C0029000400167F
:1009A00000070009000A000B000D000E000F0033C5
:1009B000003400E1001D001B0006001900050011B5
:1009C00000100036003700380028003900E000E24F
:1009D00000E30021522C002C002252500051005202
:1009E000004F0035021E021F0220022102220223B4
:1009F0000224022502260227022A0035021E021FB7
:100A000002200221022202230224022502260227BA
:100A1000024C004C003A003B003C003D003E003FD1
:100A2000002D022E022F023002310201004000414F
:100A3000004200430044004500320264024A004D77
:100A4000000100010001000100010001000100019E
:100A5000002352AB00AA00A900AE0035001E001F03
:100A6000002000210022002300240025002600276A
:100A7000002A0035001E001F002000210022002354
:100A80000024002500260027004C004C003A003BC3
:100A9000003C003D003E003F002D002E002F0030A6
:100AA0000031000100400041004200430044004585
:100AB00000320064004B004E000100010001000103
:100AC0000001002352010001000100AB00AA00A9AF
:100AD00000AE003A003B003C003D003E003F0040BD
:100AE00000410042004300440045000100007C0139
:100AF00000010001000100010001000100010001EE
:100B000000010001000100010001000100010001DD
:100B100000010001000100010001000100010001CD
:100B200000010001000100010001000100010001BD
:100B300000010001000100010001000100010001AD
:100B4000000100010001000100010001000100019D
:100B5000000100010001000100010001000100018D
:100B6000000100010001000100010001000100017D
:100B7000000100010001000100010001000100016D
:100B8000000100010001000100010001000100015D
:100B9000000100010001000100010001000100014D
:100BA000000100010001000100010001000100013D
:100BB000000100010001000100010001000100012D
:100BC000000100010001000100010001000100011D
:100BD000000100010001000100010001000100010D
:100BE00000010001000100010001000100010001FD
:100BF00000010001000100010001000100010001ED
:100C000000010001000100010001000100010001DC
:100C100000010001000100010001000100010001CC
:100C200000010001000100010001000100010001BC
:100C300000010001000100010001000100010001AC
:100C4000000100010001000100010001000100019C
:100C5000000100010001000100010001000100018C
:100C6000000100010001000100010001000100017C
:100C7000000100010001000100010001000100016C
:100C8000000100010001000100010001000100015C
:100C9000000100010001000100010001000100014C
:100CA000000100010001000100010001000100013C
:100CB000000100290A002575002F002575005D2818
:100CC0000025640020002564002000256400200029
:100CD0002564007C0025303258006D6F7573656B9C
:100CE0006579205B62746E7C782079207620685D5F
:100CF000287265702F61636C293A205B006164641F
:100D00005F6B65795F6269743A2063616E27742056
:100D10006164643A20253032580A0064656C5F6B68
:100D200065795F6269743A2063616E277420646537
:100D30006C3A20253032580A005B435D005B445D0D
:100D4000005B535D005B575D005B525D0009027400
:100D500000040100A0FA09040000010301010009D8
:100D60002111010001224400070581030800010947
:100D700004010002030000000921110100012222E8
:100D80000007058203200001070503032000010975
:100D9000040200010300000009211101000122B634
:100DA000000705840320000109040300010300007B
:100DB000000921110100012215000705850320000B
:100DC00001120100020000000854766000010001D9
:100DD000020001100330002D0053006900780074F8
:100DE00000790000001403760065006E0030006D8D
:100DF000007400720030006E00000004030904005B
:100E000011241FBECFEFDAE0DEBFCDBF12E0A0E0BD
:100E1000B1E0EAEBF6E502C005900D92A03AB10709
:100E2000D9F723E0A0EAB2E001C01D92A53BB207CA
:100E3000E1F70E94A9250C94CA2A0C940000FF93A4
:100E4000EF93E091A002F091A102309709F009958B
:100E5000EF91FF910895FC018591803011F0EFDF53
:100E6000FBCF0895FF27E0E230E247FF0CC0419539
:100E700097FF09C0EDE26095709580959095611D92
:100E8000711D811D911D27FF02C0219530E350E2A5
:100E9000AA27660F771F881F991FAA1FA41710F093
:100EA000A41B63955A95A9F7AA3008F0A95FA05D25
:100EB000AF93F395611571058105910541F7ED3209
:100EC00011F4EF93F395F21718F43F93F395FBCFDA
:100ED0008F91B5DFFA95E1F70895E991F991859140
:100EE000803021F0853219F0AADFF9CF089520E093
:100EF000E89455915532C1F3503311F468945591EB
:100F00005A3348F4505390F3220F022E220F220F2F
:100F1000200D250FF4CF0EF4219589919991533628
:100F200019F3533729F1533559F1BC018827992713
:100F3000E8945C3621F489919991689455915436DE
:100F400039F446EF7EF077FF0DC08FEF9FEF0AC0B8
:100F500055374AE039F0583540E121F0523642E049
:100F600009F00895FF93EF937DDFEF91FF91B7CFE5
:100F7000FF93EF93FC0181918030B9F360DFFBCFE9
:100F8000FF93EF9368DFF1CFDF93CF93CDB7DEB759
:100F90002596A3DFCF91DF910895482F2091B103CB
:100FA0009091780357E0291302C080E0089530E063
:100FB000529FF001539FF00D1124E758FC4F81819F
:100FC000681306C08081481303C085818111EECF6C
:100FD0002F5F3F4F2770E7CFE8EDF0E080818E7FF5
:100FE00080831092E2001092DA001092E100A0EEED
:100FF000B0E08C9181608C9380818F77808319BC65
:10100000A7EDB0E08C918E7F8C9380818F7E808362
:101010001092610308952091E4003091E50095E677
:10102000A9012091EC00822F817020FF06C08091E1
:10103000E80080FF06C080E008952091E80022FDCE
:101040001AC080916E03882389F0853089F08091E1
:10105000EB0085FD0FC02091E4003091E5004217C0
:101060005307F9F29150E1F684E0089582E0089583
:1010700083E0089581E008958091700387FF13C095
:101080008091E80082FF06C08091E8008B77809312
:10109000E80004C080916E038111F2CF0895809121
:1010A0006E038823D9F38091E80080FFF8CF809108
:1010B000E8008E77ECCF982F9093E900242F762FBD
:1010C00050E0891731F07091EC002091ED005091C3
:1010D000F00021FD07C09F5F973071F78093E90012
:1010E00081E008953091EB003E7F3093EB0030912A
:1010F000ED003D7F3093ED003091EB003160309397
:10110000EB007093EC002093ED005093F0002091E1
:10111000EE0027FDE0CF80E00895B0E0A0E0E3E935
:10112000F8E00C942A2AC8EDD0E088818F7E88836D
:10113000E7EDF0E080818160808384E082BF81E020
:101140008093610388818E7F888302EE10E0F8012E
:1011500010821092DA0081EEC82ED12CF601108296
:1011600088818F77888388818068888388818F7D54
:10117000888319BC10926E0310926F0310926D0356
:1011800010926C0390EEE92EF12CF70180818B7F99
:10119000808388818160888342E060E080E00E94F3
:1011A0005B08F60180818E7F8083F80180818160F9
:1011B0008083808188608083F70180818E7F808337
:1011C000888180618883CDB7DEB7E8E00C94462A39
:1011D000FC01809176039091770386179707A0F022
:1011E0006115710529F49091E8009E779093E800CD
:1011F00090E06115710551F4911108C08091E800EB
:1012000082FF34C080E00895BC01F2CF80916E036C
:101210008823C1F18530C1F18091E80083FD30C0A1
:101220008091E80082FDEACF8091E80080FFE1CF65
:101230008091F3002091F200382F6115710519F0AB
:101240002830310558F091E02830310509F090E060
:101250002091E8002E772093E800CBCF81918093F6
:10126000F100615071092F5F3F4FE7CF80916E030E
:10127000882341F0853041F08091E80083FFBECFA4
:1012800081E0089582E0089583E0089580916303EA
:10129000089587E797E7909301088093000888E115
:1012A0009AE00FB6F894A895809360000FBE9093D3
:1012B0006000FFCF9C014FB7F89480915A03909142
:1012C0005B03A0915C03B0915D034FBF821B930B46
:1012D00008952FB7F89460915A0370915B03809141
:1012E0005C0390915D032FBF08952FB7F894809110
:1012F0005A0390915B03A0915C03B0915D032FBFF3
:101300000895A3E0B0E0E7E8F9E00C94302A2091DA
:1013100054033091550328173907A1F090935503D2
:1013200080935403E0915203F0915303309751F0AE
:1013300024E029839B838A830084F185E02DCE01FC
:10134000019609952396E2E00C944C2AA3E0B0E0C4
:10135000ECEAF9E00C94302A2091500330915103CB
:1013600028173907A1F09093510380935003E0911F
:101370005203F0915303309751F023E029839B836C
:101380008A830084F185E02DCE010196099523968C
:10139000E2E00C944C2AE0915203F0915303309711
:1013A00029F00190F081E02D0995089580E00895DD
:1013B0008091440380FF0CC060910F0170E075952F
:1013C0006795759567956115710549F1862F0895A3
:1013D00081FF06C060910F0170E075956795F3CFAE
:1013E00060910F0182FD0BC0909143039923A1F0FE
:1013F00060910E0180910F01961738F0682F70E010
:101400006038710500F38FE70895899FC0011124AA
:1014100070E00E94FF29F4CF61E070E0D7CF81E057
:1014200008958091440380FF0DC060910D0170E02C
:10143000660F771F6038710570F56115710569F1E8
:10144000862F089581FF07C060910D0184E0689F99
:10145000B0011124EFCF82FF04C060910D0188E03C
:10146000F6CF80914503882399F020910C0160917B
:101470000D018217A0F7869FC001112433E0880F69
:10148000991F3A95E1F7622F70E00E94FF29D2CFB1
:1014900068E070E0D5CF8FE7089581E00895282FA8
:1014A00035EB2303C001112497FF04C08058910934
:1014B000892F089580589F4FFBCFF894E82FE2952D
:1014C000EF70F0E031A1282F2F7081E090E001C093
:1014D000880F2A95EAF7982F9095932391A392A1CC
:1014E000892B82A3789408959091570392FF10C09E
:1014F00041E0282F2471243009F040E031E0282F0A
:101500002871283009F030E0431711F02CE08227D1
:1015100093FF10C041E0282F2471243109F040E0EE
:1015200031E0282F2871283109F030E0431711F0FD
:101530002CE082273091580330FF10C051E0282F53
:101540002171213009F050E041E0282F2871283026
:1015500009F040E0541711F029E0822731FF10C054
:1015600041E0282F2171213109F040E031E0282F9E
:101570002871283109F030E0431711F029E0822763
:1015800094FD877E089582389105B9F1B0F48133D6
:10159000910509F47DC048F48932910509F46DC0C4
:1015A0008A32910509F47BC008958533910509F4C9
:1015B0005FC08933910509F10895833E9105D9F102
:1015C00038F4803E910529F1823E910579F1089524
:1015D000863E9105D9F1873E910509F43EC0843ECF
:1015E000910541F52091580321FF24C080915703B4
:1015F00084FD19C087EE90E0089520915703237071
:1016000009F05AC02091580323FF14C089E290E0EA
:1016100008952091570320FD38C03091580330FFC2
:1016200009C024FF43C090E080E008952091570353
:1016300022FDF7CF08952091570322FD3AC0309143
:10164000580330FD39C024FFF5CFEDCF209157036B
:1016500023FFF0CF24FDE7CFCDCF2091570323FD0B
:101660002EC03091580331FFEECF84EE90E0089504
:101670002091570325FFDECFC9CF2091570325FDC9
:1016800021C02091580323FFD5CF89E390E0D2CF2A
:101690002091570326FFCECF8AE290E00895209153
:1016A000570326FFC7CF81E390E0089583EE90E0D3
:1016B000089582EE90E0089580EE90E0089586EE21
:1016C00090E0089585E390E008951F93CF93DF9312
:1016D0000E94C30AEC01C11580E5D807F0F5C115D9
:1016E00080E4D80708F09CC0C03ED10520F5CD3C71
:1016F000D10508F082C0C83AD10578F4C53AD105C1
:1017000008F073C0C130D10519F1209709F1C43038
:10171000D105F0F4D0E0C0E01BC0C33CD105D0F748
:10172000C85AD0E0CC0FDD1FCC5BDD4F0990D881CB
:10173000C02DD4640DC0C11580E2D80708F0D1C017
:10174000C11581E0D80708F05AC0C83ED10510F78E
:10175000CE01DF91CF911F910895C03682E5D80761
:1017600018F5C03482E5D80708F06BC0C03282E5B6
:10177000D80708F05FC0C11582E5D80708F497C004
:101780002C2F2695269580E2289F900111248C2FDE
:101790008370C1E0D0E002C0CC0FDD1F8A95E2F774
:1017A000C22BD32BDD68D4CFC03A82E5D80760F4D2
:1017B000C03882E5D80708F459C0CF71D0E0DC2FDB
:1017C000CC27C46FD06AC4CFC03C82E5D80708F4E8
:1017D00062C0C03E82E5D80708F09CCFDC2FCC2742
:1017E000CC27DF71C06FD06AB3CFC55AD0E0CF5BD2
:1017F000DD4FC881D0E0D064ABCFD065A9CF8D2FAD
:101800000E94740A182FCE0199270E94C30AC12F83
:10181000D0E0DC2FCC27CC27DF71C82BD92B98CF79
:10182000CE0199270E94C30ACC27DF70C82BD92B81
:10183000D06A8ECFCF71D0E0DC2FCC27C16FD06AB9
:1018400087CF2C2F26952695277080E2289F900120
:1018500011248C2F8370C1E0D0E002C0CC0FDD1FBB
:101860008A95E2F7C22BD32BDC6872CF2C2F2695FA
:101870002695277080E2289F900111248C2F837079
:10188000C1E0D0E002C0CC0FDD1F8A95E2F7C22B89
:10189000D32BDA685DCF8C2F8F710E94740AC82F0A
:1018A000D0E0DC2FCC27CC27DF71D06251CF8C2F3A
:1018B0008F710E94740A55E0D695C7955A95E1F745
:1018C000CF70D0E0DC2FCC27282F30E084FF05C07C
:1018D00044E0220F331F4A95E1F7C22BD32BD06986
:1018E00037CF8D2F8F710E94740A182FCE01992740
:1018F0000E94C30AC12FD0E0DC2FCC27CC27DF7198
:10190000C82BD92BD2CF8095909116039823909312
:1019100016030895809116039091ED02892B909102
:10192000EC02992391F0892B90911001992371F089
:101930009091570397FF0AC09EE12CEA32E040E005
:10194000915040F441111092EC02089596E024EA7F
:1019500032E0F5CFF90151919F01552389F34F5F93
:10196000EFCF8091B10390917803981301C008954F
:101970008F5F8770FACF292F953078F58C3068F516
:1019800090E03CE0239F800D911D1124682F67702B
:1019900023E0969587952A95E1F7FC01EE0FFF1F4E
:1019A000E80FF91FE453FD4F50E040E080E0219143
:1019B00030E0062E02C0369527950A94E2F7217092
:1019C0003327042E01C0220F0A94EAF7822B4F5FBF
:1019D0005F4F4330510559F7089580E00895292F4E
:1019E000953098F58C3088F590E03CE0239F800D91
:1019F000911D1124282F277041E001C0440F2A9522
:101A0000EAF723E0969587952A95E1F7FC01EE0F1A
:101A1000FF1FE80FF91FE453FD4F30E020E070E0B6
:101A20005191DF011197CB01022E02C09695879547
:101A30000A94E2F7817081958527842385278C930A
:101A40002F5F3F4F2330310559F7089580932703C7
:101A500008959091270321E030E0F90101C0EE0FD5
:101A60008A95EAF7D90102C0AA0FBB1F6A95E2F76F
:101A7000EA2B01C0220F4A95EAF7892F8E23E8133B
:101A800005C0292B822F0E94260D08952095292319
:101A9000F9CF21E030E001C0220F8A95EAF72095C6
:101AA0008091270382230E94260D08959091EB02D6
:101AB000809589238093EB02282F277069F489177A
:101AC00059F09091580392FF07C0869586958695A8
:101AD0000E94490D1092EB02089521E030E001C010
:101AE000220F8A95EAF780912703822B0E94260D08
:101AF000089580931703089581FF03C02E9A81E013
:101B000008952E98FCCF829590E09C01220F331F00
:101B1000220F331F2C7C9595879595958795837318
:101B2000282B30E0C901880F991F8A7A35952795AF
:101B30002575822B089590911001992359F1909168
:101B4000570397FF27C0E82FE695E695E695EE3117
:101B500080F4F0E0E655FD4F282F277081E090E0FB
:101B600001C0880F2A95EAF78095928189238283A4
:101B700008959091560390FF19C01F928F938BE1A7
:101B80009DE09F938F930E94C4070F900F900F903A
:101B90000F900895E4EAF2E09191891303C0DF0108
:101BA00011971C9292E0EA3AF907B1F708959091E3
:101BB0001001992349F19091570397FF25C0E82F11
:101BC000E695E695E695EE3170F4F0E0E655FD4FCA
:101BD000877021E030E001C0220F8A95EAF7828108
:101BE000822B828308959091560390FF1EC01F920E
:101BF0008F938DEF9CE09F938F930E94C4070F906B
:101C00000F900F900F900895A4EAB2E0EFEF90E0EC
:101C10002D91821751F0EF3F19F4211101C0E92FE6
:101C20009F5F9630A9F7EF3F09F408950E2E000C40
:101C3000FF0BEE55FD4FD5CF8091560383FF96C025
:101C40008AED9CE09F938F930E94C40780914B0381
:101C50001F928F9385ED9CE09F938F930E94C40702
:101C600083ED9CE09F938F930E94C40780914C0367
:101C7000282F082E000C330B3F938F9380ED9CE0B0
:101C80009F938F930E94C4078EEC9CE09F938F9349
:101C90000E94C40780914D03282F082E000C330B9F
:101CA0003F938F938BEC9CE09F938F930E94C4078C
:101CB00089EC9CE09F938F930E94C40780914E0310
:101CC000282F082E000C330B3F938F9386EC9CE05B
:101CD0009F938F930E94C40784EC9CE09F938F9303
:101CE0000E94C40780914F03282F082E000C330B4D
:101CF0003F938F9381EC9CE09F938F930E94C40746
:101D00008EEB9CE09F938F930E94C4078DB79EB784
:101D100080960FB6F8949EBF0FBE8DBF809145038D
:101D20001F928F938BEB9CE09F938F930E94C4072D
:101D300089EB9CE09F938F930E94C407809144039A
:101D40001F928F9386EB9CE09F938F930E94C40712
:101D500083EB9CE09F938F930E94C4078DB79EB73F
:101D60000C960FB6F8949EBF0FBE8DBF0E947509EA
:101D70009C0190914C0380914D03982B21F030935E
:101D800049032093480390914E0380914F03982B71
:101D900021F03093470320934603E0915203F091E2
:101DA0005303309749F082E080934A030680F7811D
:101DB000E02D8AE493E00995089540914C039091B9
:101DC0004E0320914F03662309F469C0942B922B94
:101DD00020914D03922B31F098E09093450391E0D0
:101DE000909343038D3C41F40E94110A81958093A6
:101DF0004D030E941C0E08958E3C19F40E94110A96
:101E0000F6CF8F3C31F40E94110A819580934C03E8
:101E1000F0CF803D19F40E94110AF8CF893D29F4D2
:101E20000E94D80980934E03E4CF8A3D21F40E949A
:101E3000D8098195F7CF8B3D31F40E94D80981955F
:101E400080934F03D6CF8C3D19F40E94D809F8CF68
:101E50009FE2980F983070F4815D990B21E030E09B
:101E600001C0220F8A95EAF780914B03822B809361
:101E70004B03BFCF8D3D31F480914403816080934B
:101E80004403B7CF8E3D21F4809144038260F7CFA5
:101E90008F3D09F0AECF809144038460F0CF8D3C3C
:101EA00059F480914D0387FF0DC010924D034111ED
:101EB0000BC01092450308C08E3C81F480914D0305
:101EC00018169CF3442381F080914E0390914F03A8
:101ED000892B09F08ECF109243038BCF8F3C49F4AE
:101EE00047FFF0CF10924C0380914D038111ECCF4E
:101EF000E0CF803D19F41416ACF3E4CF893D29F40A
:101F0000191604F710924E03DDCF8A3D19F497FF9E
:101F1000D9CFF8CF8B3D29F427FFD4CF10924F03B0
:101F2000D1CF8C3D19F41216CCF3CCCF9FE2980F91
:101F3000983090F4815D990B21E030E0B90102C046
:101F4000660F771F8A95E2F7CB01809590914B033E
:101F5000892380934B03B6CF8D3D31F480914403A8
:101F60008E7F80934403AECF8E3D21F48091440355
:101F70008D7FF7CF8F3D09F0A5CF809144038B7FF4
:101F8000F0CF80910E011F928F9380910F011F92CD
:101F90008F9380910C011F928F9380910D011F925E
:101FA0008F9380910A011F928F9380910B011F9252
:101FB0008F9382ED97E09F938F930E94C4078DB714
:101FC0009EB70E960FB6F8949EBF0FBE8DBF0895B4
:101FD000883248F58E3108F07FC08B3069F130F4DB
:101FE000873009F4E0C081E399E0F1C0833109F45E
:101FF00068C08431C1F783E599E09F938F930E9475
:10200000C4070F900F9080914203882309F411C1F7
:1020100010924203109241031092400310923F032A
:1020200010923E0325C08F3409F4D6C008F03FC09B
:10203000893209F38833B9F686E599E09F938F9347
:102040000E94C4070E94C10F1F9281E08F931F92CC
:1020500088E08F938FE498E09F938F930E94C4074A
:102060008DB79EB708960FB6F8949EBF0FBE8DBF72
:1020700020914203222309F4D3C080913E03909122
:102080003F03009711F481E191E09F938F931F929A
:102090002F938FE199E09F938F930E94C4070F9035
:1020A0000F900F900F900F900F9081E00895813561
:1020B00009F4A6C008F4A6C0823509F094CF81E0E7
:1020C0008CC085E499E09F938F930E94C4070E947F
:1020D000C10F0F900F90CCCF8D518093420383306E
:1020E00009F446C078F48130E1F08230C1F11092F9
:1020F000420382E499E09F938F930E94C4070F905C
:102100000F901BC0853009F445C0D8F1863079F7AF
:102110008EE091E0909341038093400389E591E044
:1021200008C08BE091E0909341038093400385E1E8
:1021300091E090933F0380933E0380914203882374
:1021400009F496CF1F928F938EE399E09F938F931C
:102150000E94C4070F900F900F900F9089CF8AE0D4
:1021600091E090934103809340038EE191E0E1CFB1
:102170008DE091E090934103809340038AE291E0E7
:10218000D8CF8CE091E0909341038093400387E3A4
:1021900091E0CFCF8FE091E0909341038093400393
:1021A00086E491E0C6CF81E080930B0184E18093C7
:1021B0000A018AE080930D018EE180930C0188E092
:1021C00080930F0188E280930E0184E399E09F934E
:1021D0008F930E94C4077DCF8AE0E0914003F09185
:1021E00041033097D1F02081082E000C990B820F0B
:1021F000911D8F3F910541F03CF08FEF808307C028
:102200008FEFEBCF86EFE9CF97FFF8CF1082808179
:102210001F928F938BE299E099CF88E299E0D7CF14
:102220008BE199E09F938F930E94C4070F900F90CA
:102230003CCF80E008959FB7F89410925F039FBF52
:1022400090916E03943009F048C02091E9002F70FE
:102250003091EC00932F917030FD90E8922B25E0A7
:102260002093E9002091EB0020FF34C02091EE0084
:1022700027FF30C020915E03222321F02091E80047
:1022800025FF28C010925E0326E03091E80035FF5C
:1022900014C08093F1008091E80085FD27C08091F3
:1022A000E80080FFFCCF8091E8008E778093E80003
:1022B0009F709093E90080E0089530916E03343070
:1022C00049F43091EB0035FD05C0215041F481E027
:1022D00080935E039F709093E9008FEF0895EFE97C
:1022E000FFE03197F1F700C00000CFCF8FB7F8942F
:1022F00021E020935F038FBFDBCF0F931F93CF931A
:10230000DF938B01EA0190916E03943061F5809325
:10231000E9008FEF9091E800815095FD06C095EDA2
:102320009A95F1F700008111F5CF8091E80085FFC3
:102330001AC00E940B08811111C08091E80085FD30
:1023400006C08091E8008E778093E800F2CFF80114
:1023500081918F018093F100219779F78091E800B6
:102360008E778093E800DF91CF911F910F910895B0
:1023700043E050E0BC0184E00E947D11089546E0F6
:1023800050E0BC0184E00E947D11089540E250E0DD
:10239000BC0184E00E947D110895CF93DF93EC018E
:1023A00048E050E0BC0181E00E947D1188E0FE0120
:1023B000A4E6B3E001900D928A95E1F7DF91CF9109
:1023C0000895CF93C82F6FEF811164E284E290E00B
:1023D0000E94892A6FEFC11168E085E290E00E94B7
:1023E000892A6FEFC11165E286E290E00E94892A96
:1023F000CF910895CF93DF93C0E7D3E060E0CE01A3
:102400000E94892A2196C11584E0D807B9F7DF9187
:10241000CF9108951F93CF93DF93122F8730E0F46D
:102420006530D0F44C30C0F4C42FD0E0CC0FDD1FA9
:1024300098E1699FC00DD11D112498E7899FC00DB7
:10244000D11D1124632FCE0188960E94892A612F05
:10245000CE0189960E94892ADF91CF911F9108951C
:10246000AF92BF92CF92DF92EF92FF921F93CF93E2
:10247000DF938BE6C82E89E0D82ED0E07601C0E04D
:1024800014C0F50125913491412F6C2F8D2F0E949E
:102490000A1282E0A80EB11C1F5F1C3091F788E180
:1024A000E80EF11CCF5FC53019F0570110E0E9CFFD
:1024B000DF5F88E7C80ED11CD73001F7DF91CF91DD
:1024C0001F91FF90EF90DF90CF90BF90AF90089555
:1024D00080E00E94E11160E087E290E00E94892A9A
:1024E0000E9430120E94FA1181E00E94E1110895C9
:1024F00084E290E00E946B2A843289F485E290E0C5
:102500000E946B2A883059F486E290E00E946B2A80
:1025100091E0853209F090E0892F8170089580E084
:10252000FCCF0F931F93CF93DF93873030F5653047
:1025300020F54C3010F5C42FD0E0CC0FDD1F28E182
:10254000629FC00DD11D112438E7839FC00DD11D9E
:102550001124CE0188960E946B2A082F10E0102FBC
:102560000027CE0189960E946B2A9801282BC90169
:10257000DF91CF911F910F91089590E080E0F8CF07
:10258000462F753040F46C3030F4873020F4672FDC
:102590000E949112089590E080E00895CF92DF921A
:1025A000FF920F931F93CF93DF936C01009127034A
:1025B00080911703082BC6E0D0E010E0FC2EC80184
:1025C0000C2E02C0959587950A94E2F780FD0CC009
:1025D0002197A0F7F12C8F2DDF91CF911F910F91B3
:1025E000FF90DF90CF900895B6018C2F0E94C0120B
:1025F0000E94650B019761F3EECFCF93DF93EC015F
:102600000E94CE12BE010E94C0120E94650BDF9193
:10261000CF910895FC0124812223C1F08081918112
:102620000E94FD1292959F70963091F058F4925F3F
:102630009F70923058F4803F19F030F4883E30F4A7
:1026400081E008959A5FF4CF843FD1F380E008954C
:10265000883EB0F3813FD1F7F3CFA6E0B0E0E3E3EB
:10266000F3E10C942F2A49835A8349815A81992393
:10267000A1F0222391F0CA010E94CE12182F682FD8
:1026800089819A810E94EF0C69817A81812F0E9451
:10269000C0122696E3E00C944B2ACA010E94BB0CA0
:1026A000182FF2CFCF93C82F8091580382FB992720
:1026B00090F99C17F9F0C0FB82F980935803609160
:1026C00057037091580384E090E00E94A72A82E0AB
:1026D0000E94560D8091560380FF0CC01F92CF932D
:1026E00086EB92E09F938F930E94C4070F900F9008
:1026F0000F900F90CF910895EF92FF920F931F9339
:10270000CF93DF9380911001882309F469C08091F1
:10271000570387FF65C00E948A0C8093AB0240E29A
:1027200050E06EEE72E08AEA92E00E94BD2A892BA8
:1027300009F451C080E2EAEAF2E0AEEEB2E00190C4
:102740000D928A95E1F7E0915203F091530330978F
:1027500009F441C086E08093AA020480F581E02D4F
:102760008AEA92E009958091560382FF34C080FF87
:102770000EC08091AB021F928F9383ED92E09F93E6
:102780008F930E94C4070F900F900F900F90CAEA8A
:10279000D2E00DEC12E08091560380FF0BC08A81DD
:1027A0001F928F931F930F930E94C4070F900F9057
:1027B0000F900F90219682E0C83CD80761F7809176
:1027C000560380FF08C08BEC92E09F938F930E948A
:1027D000C4070F900F90CDB7DEB7E6E00C94482AFF
:1027E0000E948A0C8093A20248E050E06EE073E001
:1027F00082EA92E00E94BD2A892B69F388E0E2EA2E
:10280000F2E0AEE0B3E001900D928A95E1F7E0913D
:102810005203F09153033097F1F20280F381E02DDF
:1028200082EA92E009958091560382FFD4CF80FF1F
:102830000EC08091A2021F928F9380EF92E09F932F
:102840008F930E94C4070F900F900F900F90C2EAD1
:10285000D2E088EAE82E82E0F82E0AEE12E08091BB
:10286000560380FF0BC08A811F928F931F930F9393
:102870000E94C4070F900F900F900F902196EC16B6
:10288000FD0669F78091560380FFA5CF88EE92E0A0
:102890009CCF1092160380911001882339F180910A
:1028A000570387FF23C0ECEAF2E08EE1DF011D92BF
:1028B0008A95E9F790E080E00E94A60990E080E028
:1028C0000E9481091092ED020E947C1386E0EAE4E6
:1028D000F3E0DF011D928A95E9F71092450310920B
:1028E0004303109244030E941C0E0895E4EAF2E0B0
:1028F00086E0DCCFAAE2B0E0E0E8F4E10C942F2A15
:1029000080E793E02091F100DC012D93CD01B3E04D
:1029100088379B07B9F780917103833009F472C03F
:10292000B8F4813009F449C0823009F4B3C0809111
:10293000E80083FF91C280917003909171039A30F7
:1029400008F08AC2E92FF0E0E453F54D0C94132A05
:102950008A3009F48EC08B3009F471C0893039F7A0
:1029600080917003813219F78091740390917503FF
:10297000009711F00297D9F68091E800877F809345
:10298000E8008091E80082FF38C09091F3008091C8
:10299000F200029731F48091F100813011F086301D
:1029A00021F48091F100809363038091E8008B779C
:1029B0008093E8000E943C08BACF80917003813A6E
:1029C00009F0B5CF8091E800877F8093E80080917F
:1029D000740390917503892B61F468E084E693E0B9
:1029E00070E00E94E8088091E8008B778093E8000F
:1029F0009ECF60E090E080E0F3CF80916E03811184
:102A0000C0CF95CF80917003813A09F090CF80912B
:102A1000740390917503892B09F089CF8091E800A8
:102A2000877F8093E8008091E80080FFFCCF809151
:102A300010018093F1008091E8008E77B9CF8091EA
:102A40007003813209F073CF809174039091750304
:102A5000892B09F06CCF8091E800877F8093E80094
:102A60000E943C0880917203809310010E944914D7
:102A70005ECF80917003813209F059CF8091E800D8
:102A8000877F8093E8000E943C08809173038093C5
:102A900062034DCF80917003813A09F048CF809155
:102AA000E800877F8093E8008091E80080FFFCCFFA
:102AB00080916203BECF803899F0823809F0CCC192
:102AC000809174038F70873008F0C6C18093E9004D
:102AD0008091EB0085FB882780F91092E90006C001
:102AE00080916C0390916D03911182609091E80048
:102AF000977F9093E8008093F1001092F10080910D
:102B0000E8008E77A5C1882309F493C1823009F0CB
:102B1000A3C180917203811196C1809174038F705B
:102B20002FEF280F263008F097C18093E9002091FD
:102B3000EB0020FF88C1933031F48091EB0080627C
:102B40008093EB0080C19091EB0090619093EB003B
:102B500021E030E001C0220F8A95EAF72093EA00D5
:102B60001092EA008091EB008860EACF811174C175
:102B7000109172031F778091E3008078812B8093FE
:102B8000E3008091E800877F8093E8000E943C0882
:102B90008091E80080FFFCCF8091E3008068809303
:102BA000E30082E0111183E080936E0355C18058E9
:102BB000823008F051C120917203309173032C3D93
:102BC000E3E03E07A1F583E08A838AE289834FB779
:102BD000F894DE01139620E03EE051E2E32FF0E0AE
:102BE00050935700E49120FF03C0E295EF703F5FE0
:102BF000EF708E2F90E0EA30C0F0C7968D939D93D2
:102C00002F5F243159F74FBF8091E800877F809371
:102C1000E8006AE270E0CE0101960E94E808809127
:102C2000E8008B778093E80017C1C096E7CF8091CA
:102C3000740390917503432F55274330510509F4D0
:102C40004AC078F54130510509F47AC084E790E034
:102C5000EDE4FDE04230510509F0FEC02091E800AE
:102C6000277F2093E8002091760330917703821725
:102C7000930708F49C0140E02115310509F065C077
:102C8000411163C08091E80082FDC9CF80916E033D
:102C9000882329F2853019F28091E80083FFF2CF72
:102CA000BECF4132510509F43CC04232510509F012
:102CB000D3C08430910508F0CFC0FC01EE0FFF1F98
:102CC000E157FD4F0190F081E02D85579D4FDC01CC
:102CD0008C9190E01AC0332721303105D1F02115B5
:102CE000310561F02230310509F0B6C0E3EDFDE0B9
:102CF000E4918E2F90E0E3EDFDE007C0EBEFFDE007
:102D0000E4918E2F90E0EBEFFDE0009709F4A4C072
:102D1000A5CFE5EEFDE0E4918E2F90E0E5EEFDE03D
:102D2000F4CF8430910508F097C0880F991FFC01FB
:102D3000E956FD4F0190F081E02D89E090E08ECFC3
:102D400082E190E0E1ECFDE089CF80916E03882381
:102D500009F465CF853009F462CF8091E80083FDE6
:102D60005ECF8091E80082FD8DCF8091E80080FFEA
:102D700083CF9091F3008091F2002115310519F075
:102D80008830910550F041E0089709F040E08091CB
:102D9000E8008E778093E8006FCF44914093F10074
:102DA0003196215031090196E8CF803809F054C09E
:102DB0008091E800877F8093E80080916F03809383
:102DC000F1009DCE811148C010917203123008F0BD
:102DD00043C08091E800877F8093E80010936F03E1
:102DE0000E943C08112311F084E005C08091E300AB
:102DF00087FDFACF81E080936E0342E061EC81E0D1
:102E00000E945B0842E261EC84E00E945B0842E2BF
:102E100061EC82E00E945B0842E260EC83E00E9489
:102E20005B0842E261EC85E00E945B0880916E03E2
:102E300013C080917203813079F481E0933009F0FE
:102E400080E080936D031092E9008091E800877F15
:102E50008093E8000E943C088091E80083FF0AC04C
:102E60008091E800877F8093E8008091EB0080628A
:102E70008093EB00AA96E3E00C944B2ACF93C82FE3
:102E80001F928F9386E699E09F938F930E94C407C9
:102E900081E001C0880FCA95EAF70E94790D0E946F
:102EA00049140F900F900F900F90CF9108950E94AA
:102EB00049142FEF84E39CE0215080409040E1F7DB
:102EC00000C0000088E19AE00FB6F894A8958093BE
:102ED00060000FBE90936000FFCF882321F00E9416
:102EE000830C0E947C130895882339F09091160377
:102EF000982B909316030E947C130895882309F45D
:102F000056C0823879F40E94CB0981FF50C089E312
:102F10000E94D70D0E947C1389E30E949B0D0E94A2
:102F20007C130895833859F40E94CB0980FF3FC079
:102F300083E50E94D70D0E947C1383E5EECF843891
:102F400059F40E94CB0982FF32C087E40E94D70D5A
:102F50000E947C1387E4E1CF9CEF980F913AE8F24E
:102F600090E2980F983050F4877091E001C0990F6B
:102F70008A95EAF7892F0E94830CD1CF9BE5980FA1
:102F8000933028F490E080E00E94A609089598E527
:102F9000980F9B3128F490E080E00E948109089509
:102FA00093E3980F933118F460E00E94DD0E0895CA
:102FB000AAE0B0E0EEEDF7E10C94222A8E010F5F5B
:102FC0001F4F8AE0F80111928A95E9F79AE7E92EF6
:102FD00092E0F92E68012FE7422E22E0522E66245D
:102FE0006394712C4BE8842E42E0942EF70181917A
:102FF0007F018F3F09F445C0F894E82FE295EF7008
:10300000F0E021A18F70A30102C0440F551F8A95E3
:10301000E2F7CA01922F982B91A392A18095892360
:1030200082A3789400C0EFE7F2E021E030E0B12C19
:10303000A12C41914F3F09F44BC0A42FA295AF7032
:10304000B0E090968C9190E04F7002C09595879576
:103050004A95E2F780FD3CC0C901A82AB92A220F8F
:10306000331F8E169F0629F7F701319780818F3F16
:1030700011F00E945D0A50EA5A95F1F7F601B1820B
:10308000A082F2E0CF0ED11C4E145F0409F0AECF47
:103090004AE050E0B8018DE193E00E94BD2A892BFF
:1030A000E1F08AE0F801ADE1B3E001900D928A957C
:1030B000E1F781E080931C030E94750990931B0344
:1030C00080931A0310E0812F2A96E0E10C943E2AA7
:1030D00090E080E0C2CF10E01FC010911C031123CC
:1030E00089F380911A0390911B030E945A09059756
:1030F00048F34AE050E06DE173E083E393E00E941F
:10310000BD2A892B41F38AE0EDE1F3E0A3E3B3E0CC
:1031100001900D928A95E1F710921C03D4CFA8E09C
:10312000B0E0E5E9F8E10C94302A65EE7EEF90E03E
:1031300080E00E94A72A60E082E090E00E94892A55
:1031400081E08093170361E083E090E00E94892A88
:1031500060E074E184E090E00E94A72A60E086E0ED
:1031600090E00E94892A60E087E090E00E94892A2E
:1031700040E050E0BA0188E090E00E949B2A60E0C5
:1031800083E290E00E94892A60E08CE090E00E9457
:10319000892A60E08DE090E00E94892A19821A82D3
:1031A0001B821C821D821E821F82188648E050E00E
:1031B00067E170E0CE0101960E94792A40E050E07C
:1031C000BA018FE190E00E949B2A80E00E94E11109
:1031D0000E94681240E050E0BA018FE090E00E9447
:1031E0009B2A40E050E0BA0183E190E00E949B2AD4
:1031F0002896E2E00C944C2AB0E0A0E0E2E0F9E18D
:103200000C942B2AEBEFE80FEF3308F062C1F0E0EB
:10321000EA52F54D0C94132A83E090E00E946B2A49
:103220001F928F938EE994E09F938F930E94C4071F
:1032300082E090E00E946B2A83FB992790F91F920D
:103240009F9382FB992790F91F929F9381FB992767
:1032500090F91F929F93982F91701F929F931F92A6
:103260008F9385E594E09F938F930E94C40784E039
:1032700090E00E94732A93FB222720F91F922F933C
:1032800087FB222720F91F922F9386FB222720F904
:103290001F922F9385FB222720F91F922F9384FBE7
:1032A000222720F91F922F9383FB222720F91F92B8
:1032B0002F9382FB222720F91F922F9391FB222725
:1032C00020F91F922F93292F21701F922F9381FB9A
:1032D000222720F91F922F93282F21701F922F93BE
:1032E0009F938F9386E593E09F938F930E94C407EB
:1032F0008DB79EB78A960FB6F8949EBF0FBE8DBF4E
:1033000081E02AC081EC97E09F938F930E94C407CD
:103310000E948F180F900F90F3CF8BEB94E09F9348
:103320008F930E94C407F6CF80915603807F8093CD
:10333000560380E796E09F938F930E94C4078DEB1E
:1033400097E09F938F930E94C40781E080933D0391
:103350000F900F900F900F90CDB7DEB7E7E00C9471
:10336000472A81EA97E09F938F930E94C4070E94A7
:1033700049149FEF24E38CE0915020408040E1F716
:1033800000C000000E94490990915603892F8E7F4A
:1033900090FF81608093560380FF03C085E997E02A
:1033A000BECF88E897E09F938F930E94C4078091D7
:1033B0005603817F80935603ADCF90915603892F9A
:1033C0008D7F91FF82608093560381FF0AC08BE757
:1033D00097E09F938F930E94C4078091560381606A
:1033E000E9CF8DE697E09BCF90915603892F8B7F95
:1033F00092FF84608093560382FF03C08EE597E0BE
:10340000E8CF8EE497E08BCF90915603892F877F8A
:1034100093FF88608093560383FF03C082E497E0A4
:10342000D8CF85E397E07BCF8EE691E09F938F9393
:1034300087E996E09F938F930E94C4070F900F90A7
:103440000F900F905DCF0E946909062FF72EE82E8E
:10345000D92EC0915703C7FBCC27C0F91091620346
:10346000D09110010E94CB09DF92EF92FF920F934F
:103470001F92CF931F921F931F92DF931F928F93E0
:103480008AE996E09F938F930E94C4078DB79EB7F9
:103490000E960FB6F8949EBF0FBE8DBF31CF0E941F
:1034A000491490915703892F97FB87F9805880938F
:1034B000570387FF03C08BE297E031CF80E297E0AC
:1034C0002ECF80E00E943E171BCF8953FBCF8D513A
:1034D000F9CF8EE197E09F938F930E94C4070F90DE
:1034E0000F9080E039CFCF93C82F8823C9F082385E
:1034F000C9F40E94CB0981FD13C089E30E94D70D56
:103500000E947C132FEF87EE93E021508040904083
:10351000E1F700C0000089E30E949B0D0E947C132C
:10352000CF9108958338A1F40E94CB0980FDF8CF94
:1035300083E50E94D70D0E947C132FEF81EE94E06B
:10354000215080409040E1F700C0000083E5E4CFC7
:103550008438A1F40E94CB0982FDE2CF87E40E9467
:10356000D70D0E947C132FEF81EE94E02150804014
:103570009040E1F700C0000087E4CECF8CEF8C0FC5
:10358000813A08F084C080913D038130B9F18823ED
:1035900059F1823009F468C010923D038091100106
:1035A000882309F465C08091570387FF61C0EC2F21
:1035B000E695E695E695F0E0E655FD4F828190E0D0
:1035C0004C2F477021E030E002C0220F331F4A9594
:1035D000E2F782239323892B09F455C08C2F0E9494
:1035E0009B0D0E947C134FC0809116038232B1F66E
:1035F0008C2F0E94FC18811193CFD0CF809116039D
:103600008232B1F3C43129F168F4CB3079F0C031A2
:1036100021F180EB92E09F938F930E94C4070F905B
:103620000F9019C0C932A9F0C83399F780E796E026
:103630009F938F930E94C40782EB92E09F938F9396
:103640000E94C4070F900F900F900F9081E081703F
:10365000D2CF10923D0380E0FACF82E080933D0309
:1036600088E30E94E80FF2CF8C2F0E94E80F58CF1A
:10367000E4EAF2E08AEA92E02191C21709F4AECFBF
:103680008E179F07C9F78C2F0E94D70D47CF80E276
:103690008C0F883068F4C77021E030E001C0220F41
:1036A000CA95EAF780911603822B8093160336CFD2
:1036B000EBE5EC0FE33040F4F0E0EF5BFD4F808191
:1036C00090E00E94A6092CCFE8E5EC0FEB3150F416
:1036D000F0E0EE0FFF1FEC5BFD4F808191810E94B7
:1036E00081091ECF83E38C0F833108F019CF61E08D
:1036F0008C2F0E94DD0E14CF1F93CF93DF93182FD2
:10370000EB010E94731A209739F4812F0E947E17D3
:10371000DF91CF911F9108958FE99FE00197F1F715
:1037200000C000002197EFCF0F931F93CF93DF933B
:10373000C62FD42F022FFC0185818823A9F0609326
:10374000B4030E9475099093B3038093B203C770CA
:1037500081E001C0880FCA95EAF70E947417DF91D3
:10376000CF911F910F9108958091B403681334C0D5
:103770008091B2039091B3030E945A09883C91054D
:1037800058F510E21D0FCD17B9F080E28C0F88308C
:1037900040F4C77081E001C0880FCA95EAF70E9423
:1037A0006D17183048F481E09D2F977001C0880F85
:1037B0009A95EAF70E94741770E060E0802F0E94EB
:1037C0007C1B183060F6D77081E001C0880FDA9555
:1037D000EAF70E946D17C3CFC77081E001C0880F60
:1037E000CA95EAF7F6CFA8E0B0E0E9EFFBE10C9468
:1037F000222A8C01DC0114968C911497882309F4F9
:10380000BEC021E04C9111965C91119712966C917B
:10381000129713967C91139715969C910E942D13E5
:103820007C01F8018581882309F448C1C7019757B5
:103830008038910508F01CC5FFE0FE1508F48FC024
:103840008FEF93E00E946B2A811189C060E7A62E5A
:1038500063E0B62EE1104DC0FE01339686E0DF0135
:103860001D928A95E9F75AE0452E7501BFEFEB1AD4
:10387000FB0AC5010E946B2A89831A82882309F4F6
:103880006EC0813009F07FC06501E2E0CE0ED11C30
:10389000C7010E946B2A8A83882309F460C09FEFC6
:1038A000980F9330A0F5F3E0AF0EB11CC6010E9453
:1038B0006B2A8B83882309F452C01C82DE01119687
:1038C0007D01F7012081222381F2213009F09DC082
:1038D00091818281913009F058C0F2E0EF0EF11C25
:1038E00070E060E0893311F460E570E00E947C1BB9
:1038F00053C0A11424E0B20691F1C5010E946B2AC5
:10390000811101C0EA943FEFA31AB30AA3CF560175
:103910008430A1F642E0E42EF12C56012FEFA21ADA
:10392000B20AC6010E946B2AE1E0F0E0EC0FFD1F35
:10393000EE0DFF1D8083882391F08C3741F4E2E087
:10394000F0E0EC0FFD1FEE0DFF1D1082B7CF3FEF33
:10395000E31AF30A650187E0E816F104F1F68091B5
:10396000EB02877061F0D80115968C91882339F0AD
:103970008091580382FF03C082E00E94560D289672
:10398000E0E10C943E2A570199CF923049F422E0AD
:10399000E20EF11C0E94731A9FEFE91AF90A91CF07
:1039A000933031F432E0E30EF11C0E947E17F4CF25
:1039B000943021F08FEFE81AF80AEECF92E0E90E8A
:1039C000F11C30E020E0B7016F5F7F4FD701119607
:1039D0004C918053990B8A30910560F02115310587
:1039E000D9F2EFE9FFE03197F1F700C00000215074
:1039F0003109F4CF429EF001439EF00D11249C0149
:103A00002E0F3F1F842F7B01DECFE22FF0E0E35F1C
:103A1000FD4F5490822F86958695869590E0FC0107
:103A2000E350FE4F64902770712C022E02C07594F3
:103A300067940A94E2F7F1E06F227724FC01E351E6
:103A4000FE4F8490912C022E02C0959487940A9484
:103A5000E2F731E083229924FC01E352FE4FC49047
:103A6000D12C02C0D594C7942A95E2F781E0C822F0
:103A7000DD246114710419F081EE0E94731A81141F
:103A8000910419F086EE0E94731A70E060E0852DB3
:103A90000E947C1B8114910419F086EE0E947E170F
:103AA0006114710419F081EE0E947E17C114D104D3
:103AB00009F472CF70E060E08CE218CFF701E851B2
:103AC000FC47E730F10508F0C6C3EB5EF44D0C94FB
:103AD000132A26E241EE61EEC8010E94941B3FCFFB
:103AE00027E245EE65EEF8CF26E241EE60EEF4CF38
:103AF00027E245EE64EEF0CF26E241EE62EEECCF37
:103B000027E245EE66EEE8CF28E241E0EBCF809178
:103B1000570381608093570395C080915803886054
:103B2000809358038FC0809157038260F3CF8091B8
:103B300057038460EFCF809157038860EBCF80916B
:103B400058038160EDCF809158038260E9CF809166
:103B500057038061DFCF809157038062DBCF809174
:103B600057038064D7CF0E9449148091570380681F
:103B7000D1CF809157038C60CDCF80915803836063
:103B8000CFCF809157038E7FC5CF80915803877F19
:103B9000C7CF809157038D7FBDCF809157038B7F17
:103BA000B9CF80915703877FB5CF809158038E7F1F
:103BB000B7CF809158038D7FB3CF809157038F7E0D
:103BC000A9CF809157038F7DA5CF809157038F7B1D
:103BD000A1CF0E944914809157038F779BCF80918A
:103BE0005703837F97CF809158038C7F99CF809123
:103BF000570382FB992790F921E0922790FB82F9E5
:103C000090FB83F987CF80915803982F90959170FE
:103C10008E7F892B90FB81F983CF90915703892F59
:103C20008F7B96FF806476CF0E9449149091570352
:103C3000892F97FB87F980586DCF61E08EE090E087
:103C40000E94892A609157037091580384E090E0A4
:103C50000E94A72A0E94491482CE60E0EFCF909183
:103C60005703892F8F7E94FF806154CF9091570323
:103C7000892F8E7F90FF81604DCF90915803892FBF
:103C8000877F93FF88604CCF85E3E0C285E3EDC278
:103C9000A7E7EA16ACE7FA0609F470C082E0B8E7D5
:103CA000EB16BCE7FB0609F46AC0E3E0EE16ECE7AE
:103CB000FE0609F4A6C008F06EC021E0E2162CE76B
:103CC000F20609F4A4C008F086C0E1148CE7F806F7
:103CD00009F474C0F8018581E080F180882309F43B
:103CE000A4C0C7010E94CE12D82E682FC7010E941F
:103CF000EF0CB7018D2D0E94C0120E94650B7C0154
:103D0000882ED8011596AC90159716969C90929493
:103D10003FE093228091EB02877009F1DA2CAA2010
:103D2000F9F08F2D807F803469F080E28E0D88302D
:103D3000B0F08F2D807E803229F4B1E0BE1578F48A
:103D4000992069F08091580382FF09C082E00E94A7
:103D5000560D8091EB028770DD24D3948111D12C14
:103D6000CF2CC2942FE0C222EBE0EC1508F4C5C0C2
:103D7000EC2DF0E0E45EF44D0C94132A81E00E94F7
:103D80006D0D43E062E081E00E94290DE8CD81E005
:103D90000E94490DF6CF9BE5E9169CE7F90609F468
:103DA00042C0ACE5EA16ACE7FA0699F1BAE5EB16C3
:103DB000BCE7FB0609F08ECF81E032C00E944914B7
:103DC000EFEFF4E32CE0E150F0402040E1F700C0D9
:103DD00000000E94490990915603892F8E7F90FF21
:103DE00081608093560380FF09C08FE992E09F9322
:103DF0008F930E94C4070F900F90B1CD8DE892E091
:103E0000F6CF6FEF7FEF90E080E00E94A72A0E943C
:103E100057178091580382FB882780F991E0892702
:103E20000E94521357CF80E0FBCFC7010E94BB0C0A
:103E3000D82E5FCFFF2DFF70BF2E8F2D807F19F002
:103E4000B29490EFB922AA20B9F0BB2069F080E2C9
:103E50008E0D883010F0811009C080911603B82AA9
:103E6000B09216030E947C138E2D45C08091ED0206
:103E7000B82AB092ED02F6CF8E2D0E947E17BB209D
